 getvern001

 Timestamp is 8ccbaeed (reproducible build file hash)

 Preferred load address is 0000000180000000

 Start         Length     Name                   Class
 0001:00000000 00002ad0H .text$mn                CODE
 0001:00002ad0 00000036H .text$mn$00             CODE
 0001:00002b06 00000092H .text$x                 CODE
 0002:00000000 00000198H .idata$5                DATA
 0002:00000198 00000038H .00cfg                  DATA
 0002:000001d0 00000008H .CRT$XCA                DATA
 0002:000001d8 00000008H .CRT$XCZ                DATA
 0002:000001e0 00000008H .CRT$XIA                DATA
 0002:000001e8 00000008H .CRT$XIC                DATA
 0002:000001f0 00000008H .CRT$XIZ                DATA
 0002:000001f8 00000008H .CRT$XLA                DATA
 0002:00000200 00000008H .CRT$XLZ                DATA
 0002:00000208 00000008H .CRT$XPA                DATA
 0002:00000210 00000008H .CRT$XPZ                DATA
 0002:00000218 00000008H .CRT$XTA                DATA
 0002:00000220 00000010H .CRT$XTZ                DATA
 0002:00000228 00000000H .gehcont$y              DATA
 0002:00000228 00000000H .gfids$y                DATA
 0002:00000230 00001ad0H .rdata                  DATA
 0002:00001d00 00000000H .rdata$CastGuardVftablesA DATA
 0002:00001d00 00000000H .rdata$CastGuardVftablesC DATA
 0002:00001d00 00000028H .rdata$T                DATA
 0002:00001d28 000000a4H .rdata$voltmd           DATA
 0002:00001dcc 0000031cH .rdata$zzzdbg           DATA
 0002:000020e8 00000008H .rtc$IAA                DATA
 0002:000020f0 00000008H .rtc$IZZ                DATA
 0002:000020f8 00000008H .rtc$TAA                DATA
 0002:00002100 00000008H .rtc$TZZ                DATA
 0002:00002108 00000004H .tls                    DATA
 0002:0000210c 00000004H .tls$                   DATA
 0002:00002110 00000008H .tls$ZZZ                DATA
 0002:00002118 000002d8H .xdata                  DATA
 0002:000023f0 000003a0H .edata                  DATA
 0002:00002790 00000064H .idata$2                DATA
 0002:000027f4 00000014H .idata$3                DATA
 0002:00002808 00000198H .idata$4                DATA
 0002:000029a0 0000041eH .idata$6                DATA
 0003:00000000 00000080H .data                   DATA
 0003:00000080 0001b238H .bss                    DATA
 0004:00000000 00000378H .pdata                  DATA

  Address         Publics by Value              Rva+Base               Lib:Object

 0000:00000000       __AbsoluteZero             0000000000000000     <absolute>
 0000:00000000       ___safe_se_handler_count   0000000000000000     <absolute>
 0000:00000000       ___safe_se_handler_table   0000000000000000     <absolute>
 0000:00000000       __arm64x_extra_rfe_table   0000000000000000     <absolute>
 0000:00000000       __arm64x_extra_rfe_table_size 0000000000000000     <absolute>
 0000:00000000       __arm64x_native_entrypoint 0000000000000000     <absolute>
 0000:00000000       __arm64x_redirection_metadata 0000000000000000     <absolute>
 0000:00000000       __arm64x_redirection_metadata_count 0000000000000000     <absolute>
 0000:00000000       __dynamic_value_reloc_table 0000000000000000     <absolute>
 0000:00000000       __enclave_config           0000000000000000     <absolute>
 0000:00000000       __guard_check_icall_a64n_fptr 0000000000000000     <absolute>
 0000:00000000       __guard_eh_cont_count      0000000000000000     <absolute>
 0000:00000000       __guard_eh_cont_table      0000000000000000     <absolute>
 0000:00000000       __guard_fids_count         0000000000000000     <absolute>
 0000:00000000       __guard_fids_table         0000000000000000     <absolute>
 0000:00000000       __guard_iat_count          0000000000000000     <absolute>
 0000:00000000       __guard_iat_table          0000000000000000     <absolute>
 0000:00000000       __guard_longjmp_count      0000000000000000     <absolute>
 0000:00000000       __guard_longjmp_table      0000000000000000     <absolute>
 0000:00000000       __hybrid_auxiliary_iat     0000000000000000     <absolute>
 0000:00000000       __hybrid_auxiliary_iat_copy 0000000000000000     <absolute>
 0000:00000000       __hybrid_code_map          0000000000000000     <absolute>
 0000:00000000       __hybrid_code_map_count    0000000000000000     <absolute>
 0000:00000000       __x64_code_ranges_to_entry_points 0000000000000000     <absolute>
 0000:00000000       __x64_code_ranges_to_entry_points_count 0000000000000000     <absolute>
 0000:00000100       __guard_flags              0000000000000100     <absolute>
 0000:00000000       __ImageBase                0000000180000000     <linker-defined>
 0001:00000000       ?NewObject@JNIEnv_@@QEAAPEAV_jobject@@PEAV_jclass@@PEAU_jmethodID@@ZZ 0000000180001000 f i libgetvern001.obj
 0001:00000028       ?TranslateError@@YAPEBDW4jvmtiError@@@Z 0000000180001028 f   libgetvern001.obj
 0001:000002e0       ?nsk_jni_check_exception@@YAHPEAUJNIEnv_@@QEBDH@Z 00000001800012e0 f   libgetvern001.obj
 0001:00000424       ?nsk_jni_lverify@@YAHHPEAUJNIEnv_@@HQEBDH1ZZ 0000000180001424 f   libgetvern001.obj
 0001:000004c4       Agent_Initialize           00000001800014c4 f   libgetvern001.obj
 0001:00000538       Agent_OnAttach             0000000180001538 f   libgetvern001.obj
 0001:00000538       Agent_OnLoad               0000000180001538 f   libgetvern001.obj
 0001:00000540       Java_nsk_jvmti_GetVersionNumber_getvern001_check 0000000180001540 f   libgetvern001.obj
 0001:00000668       Java_nsk_jvmti_unit_FollowReferences_FollowRefObjects_addRefToVerify 0000000180001668 f   libgetvern001.obj
 0001:00000840       Java_nsk_jvmti_unit_FollowReferences_FollowRefObjects_getTag 0000000180001840 f   libgetvern001.obj
 0001:00000900       Java_nsk_jvmti_unit_FollowReferences_FollowRefObjects_resetRefsToVerify 0000000180001900 f   libgetvern001.obj
 0001:00000908       Java_nsk_jvmti_unit_FollowReferences_FollowRefObjects_resetTags 0000000180001908 f   libgetvern001.obj
 0001:0000094c       Java_nsk_jvmti_unit_FollowReferences_FollowRefObjects_setTag 000000018000194c f   libgetvern001.obj
 0001:00000ba4       Java_nsk_share_jvmti_ArgumentHandler_getAgentOptionsString 0000000180001ba4 f   libgetvern001.obj
 0001:00000c54       Java_nsk_share_jvmti_DebugeeClass_checkStatus 0000000180001c54 f   libgetvern001.obj
 0001:00000cdc       Java_nsk_share_jvmti_DebugeeClass_resetAgentData 0000000180001cdc f   libgetvern001.obj
 0001:00000d3c       Java_nsk_share_jvmti_RedefineAgent_agentStatus 0000000180001d3c f   libgetvern001.obj
 0001:00000d48       Java_nsk_share_jvmti_RedefineAgent_isRedefined 0000000180001d48 f   libgetvern001.obj
 0001:00000d54       Java_nsk_share_jvmti_RedefineAgent_redefineAttempted 0000000180001d54 f   libgetvern001.obj
 0001:00000d60       MA_checkStatus             0000000180001d60 f   libgetvern001.obj
 0001:00000e04       __local_stdio_printf_options 0000000180001e04 f i libgetvern001.obj
 0001:00000fe4       exitOnError                0000000180001fe4 f   libgetvern001.obj
 0001:00001098       fprintf                    0000000180002098 f i libgetvern001.obj
 0001:000010dc       nsk_jvmti_lverify          00000001800020dc f   libgetvern001.obj
 0001:000011cc       nsk_jvmti_resetAgentData   00000001800021cc f   libgetvern001.obj
 0001:0000124c       nsk_jvmti_setFailStatus    000000018000224c f   libgetvern001.obj
 0001:00001288       nsk_lcomplain              0000000180002288 f   libgetvern001.obj
 0001:000012a8       nsk_ldisplay               00000001800022a8 f   libgetvern001.obj
 0001:000012c8       nsk_ltrace                 00000001800022c8 f   libgetvern001.obj
 0001:000012e8       nsk_lvcomplain             00000001800022e8 f   libgetvern001.obj
 0001:000014a0       nsk_lvdisplay              00000001800024a0 f   libgetvern001.obj
 0001:000014ec       nsk_lverify                00000001800024ec f   libgetvern001.obj
 0001:00001548       nsk_lvtrace                0000000180002548 f   libgetvern001.obj
 0001:000015a8       nsk_printf                 00000001800025a8 f   libgetvern001.obj
 0001:000015d0       nsk_vprintf                00000001800025d0 f   libgetvern001.obj
 0001:00001684       printf                     0000000180002684 f i libgetvern001.obj
 0001:00001bac       __raise_securityfailure    0000000180002bac f   MSVCRT:gs_report.obj
 0001:00001be0       __report_gsfailure         0000000180002be0 f   MSVCRT:gs_report.obj
 0001:00001e20       __GSHandlerCheck           0000000180002e20 f   MSVCRT:gshandler.obj
 0001:00001e40       __GSHandlerCheckCommon     0000000180002e40 f   MSVCRT:gshandler.obj
 0001:00001eb0       __security_check_cookie    0000000180002eb0 f   MSVCRT:amdsecgs.obj
 0001:000021f0       _DllMainCRTStartup         00000001800031f0 f   MSVCRT:dll_dllmain.obj
 0001:00002230       __scrt_acquire_startup_lock 0000000180003230 f   MSVCRT:utility.obj
 0001:0000226c       __scrt_dllmain_after_initialize_c 000000018000326c f   MSVCRT:utility.obj
 0001:000022a0       __scrt_dllmain_before_initialize_c 00000001800032a0 f   MSVCRT:utility.obj
 0001:000022b8       __scrt_dllmain_crt_thread_attach 00000001800032b8 f   MSVCRT:utility.obj
 0001:000022e0       __scrt_dllmain_crt_thread_detach 00000001800032e0 f   MSVCRT:utility.obj
 0001:000022f8       __scrt_dllmain_exception_filter 00000001800032f8 f   MSVCRT:utility.obj
 0001:00002358       __scrt_dllmain_uninitialize_c 0000000180003358 f   MSVCRT:utility.obj
 0001:00002388       __scrt_dllmain_uninitialize_critical 0000000180003388 f   MSVCRT:utility.obj
 0001:0000239c       __scrt_initialize_crt      000000018000339c f   MSVCRT:utility.obj
 0001:000023e8       __scrt_initialize_onexit_tables 00000001800033e8 f   MSVCRT:utility.obj
 0001:00002474       __scrt_is_nonwritable_in_current_image 0000000180003474 f   MSVCRT:utility.obj
 0001:0000250c       __scrt_release_startup_lock 000000018000350c f   MSVCRT:utility.obj
 0001:00002530       __scrt_uninitialize_crt    0000000180003530 f   MSVCRT:utility.obj
 0001:0000255c       _onexit                    000000018000355c f   MSVCRT:utility.obj
 0001:00002598       atexit                     0000000180003598 f   MSVCRT:utility.obj
 0001:000025b0       __crt_debugger_hook        00000001800035b0 f   MSVCRT:utility_desktop.obj
 0001:000025b8       __scrt_fastfail            00000001800035b8 f   MSVCRT:utility_desktop.obj
 0001:00002704       _guard_check_icall_nop     0000000180003704 f i MSVCRT:guard_support.obj
 0001:00002708       __security_init_cookie     0000000180003708 f   MSVCRT:gs_support.obj
 0001:000027b4       DllMain                    00000001800037b4 f   MSVCRT:dll_dllmain_stub.obj
 0001:000027d8       ?__scrt_initialize_type_info@@YAXXZ 00000001800037d8 f   MSVCRT:tncleanup.obj
 0001:000027e8       ?__scrt_uninitialize_type_info@@YAXXZ 00000001800037e8 f   MSVCRT:tncleanup.obj
 0001:000027f4       __local_stdio_scanf_options 00000001800037f4 f i MSVCRT:default_local_stdio_options.obj
 0001:000027fc       __scrt_initialize_default_local_stdio_options 00000001800037fc f   MSVCRT:default_local_stdio_options.obj
 0001:00002818       __scrt_get_dyn_tls_init_callback 0000000180003818 f   MSVCRT:dyn_tls_init.obj
 0001:00002820       _RTC_Initialize            0000000180003820 f   MSVCRT:initsect.obj
 0001:0000285c       _RTC_Terminate             000000018000385c f   MSVCRT:initsect.obj
 0001:00002898       __isa_available_init       0000000180003898 f   MSVCRT:cpu_disp.obj
 0001:00002a44       _get_startup_argv_mode     0000000180003a44 f   MSVCRT:argv_mode.obj
 0001:00002a4c       __scrt_is_ucrt_dll_in_use  0000000180003a4c f   MSVCRT:ucrt_detection.obj
 0001:00002a60       memcpy                     0000000180003a60 f   vcruntime:VCRUNTIME140.dll
 0001:00002a66       memset                     0000000180003a66 f   vcruntime:VCRUNTIME140.dll
 0001:00002a6c       strchr                     0000000180003a6c f   vcruntime:VCRUNTIME140.dll
 0001:00002a72       __C_specific_handler       0000000180003a72 f   vcruntime:VCRUNTIME140.dll
 0001:00002a78       __std_type_info_destroy_list 0000000180003a78 f   vcruntime:VCRUNTIME140.dll
 0001:00002a7e       strcmp                     0000000180003a7e f   ucrt:api-ms-win-crt-string-l1-1-0.dll
 0001:00002a84       strlen                     0000000180003a84 f   ucrt:api-ms-win-crt-string-l1-1-0.dll
 0001:00002a8a       _initterm                  0000000180003a8a f   ucrt:api-ms-win-crt-runtime-l1-1-0.dll
 0001:00002a90       _initterm_e                0000000180003a90 f   ucrt:api-ms-win-crt-runtime-l1-1-0.dll
 0001:00002a96       _seh_filter_dll            0000000180003a96 f   ucrt:api-ms-win-crt-runtime-l1-1-0.dll
 0001:00002a9c       _configure_narrow_argv     0000000180003a9c f   ucrt:api-ms-win-crt-runtime-l1-1-0.dll
 0001:00002aa2       _initialize_narrow_environment 0000000180003aa2 f   ucrt:api-ms-win-crt-runtime-l1-1-0.dll
 0001:00002aa8       _initialize_onexit_table   0000000180003aa8 f   ucrt:api-ms-win-crt-runtime-l1-1-0.dll
 0001:00002aae       _register_onexit_function  0000000180003aae f   ucrt:api-ms-win-crt-runtime-l1-1-0.dll
 0001:00002ab4       _execute_onexit_table      0000000180003ab4 f   ucrt:api-ms-win-crt-runtime-l1-1-0.dll
 0001:00002aba       _crt_atexit                0000000180003aba f   ucrt:api-ms-win-crt-runtime-l1-1-0.dll
 0001:00002ac0       _cexit                     0000000180003ac0 f   ucrt:api-ms-win-crt-runtime-l1-1-0.dll
 0001:00002ac8       __acrt_initialize          0000000180003ac8 f   MSVCRT:ucrt_stubs.obj
 0001:00002ac8       __acrt_thread_attach       0000000180003ac8 f   MSVCRT:ucrt_stubs.obj
 0001:00002ac8       __acrt_thread_detach       0000000180003ac8 f   MSVCRT:ucrt_stubs.obj
 0001:00002ac8       __acrt_uninitialize        0000000180003ac8 f   MSVCRT:ucrt_stubs.obj
 0001:00002ac8       __acrt_uninitialize_critical 0000000180003ac8 f   MSVCRT:ucrt_stubs.obj
 0001:00002ac8       __scrt_stub_for_acrt_initialize 0000000180003ac8 f   MSVCRT:ucrt_stubs.obj
 0001:00002ac8       __scrt_stub_for_acrt_thread_attach 0000000180003ac8 f   MSVCRT:ucrt_stubs.obj
 0001:00002ac8       __scrt_stub_for_acrt_thread_detach 0000000180003ac8 f   MSVCRT:ucrt_stubs.obj
 0001:00002ac8       __scrt_stub_for_acrt_uninitialize 0000000180003ac8 f   MSVCRT:ucrt_stubs.obj
 0001:00002ac8       __scrt_stub_for_acrt_uninitialize_critical 0000000180003ac8 f   MSVCRT:ucrt_stubs.obj
 0001:00002ac8       __vcrt_initialize          0000000180003ac8 f   MSVCRT:ucrt_stubs.obj
 0001:00002ac8       __vcrt_thread_attach       0000000180003ac8 f   MSVCRT:ucrt_stubs.obj
 0001:00002ac8       __vcrt_thread_detach       0000000180003ac8 f   MSVCRT:ucrt_stubs.obj
 0001:00002ac8       __vcrt_uninitialize        0000000180003ac8 f   MSVCRT:ucrt_stubs.obj
 0001:00002ac8       __vcrt_uninitialize_critical 0000000180003ac8 f   MSVCRT:ucrt_stubs.obj
 0001:00002acc       __scrt_stub_for_is_c_termination_complete 0000000180003acc f   MSVCRT:ucrt_stubs.obj
 0001:00002acc       _is_c_termination_complete 0000000180003acc f   MSVCRT:ucrt_stubs.obj
 0001:00002ae0       _guard_dispatch_icall_nop  0000000180003ae0 f   MSVCRT:guard_dispatch.obj
 0001:00002b00       _guard_xfg_dispatch_icall_nop 0000000180003b00 f   MSVCRT:guard_xfg_dispatch.obj
 0002:00000000       __imp_RtlCaptureContext    0000000180004000     kernel32:KERNEL32.dll
 0002:00000008       __imp_RtlLookupFunctionEntry 0000000180004008     kernel32:KERNEL32.dll
 0002:00000010       __imp_RtlVirtualUnwind     0000000180004010     kernel32:KERNEL32.dll
 0002:00000018       __imp_UnhandledExceptionFilter 0000000180004018     kernel32:KERNEL32.dll
 0002:00000020       __imp_SetUnhandledExceptionFilter 0000000180004020     kernel32:KERNEL32.dll
 0002:00000028       __imp_GetCurrentProcess    0000000180004028     kernel32:KERNEL32.dll
 0002:00000030       __imp_TerminateProcess     0000000180004030     kernel32:KERNEL32.dll
 0002:00000038       __imp_IsProcessorFeaturePresent 0000000180004038     kernel32:KERNEL32.dll
 0002:00000040       __imp_CloseHandle          0000000180004040     kernel32:KERNEL32.dll
 0002:00000048       __imp_InitializeCriticalSectionAndSpinCount 0000000180004048     kernel32:KERNEL32.dll
 0002:00000050       __imp_DeleteCriticalSection 0000000180004050     kernel32:KERNEL32.dll
 0002:00000058       __imp_CreateEventW         0000000180004058     kernel32:KERNEL32.dll
 0002:00000060       __imp_GetModuleHandleW     0000000180004060     kernel32:KERNEL32.dll
 0002:00000068       __imp_GetProcAddress       0000000180004068     kernel32:KERNEL32.dll
 0002:00000070       __imp_IsDebuggerPresent    0000000180004070     kernel32:KERNEL32.dll
 0002:00000078       __imp_QueryPerformanceCounter 0000000180004078     kernel32:KERNEL32.dll
 0002:00000080       __imp_GetCurrentProcessId  0000000180004080     kernel32:KERNEL32.dll
 0002:00000088       __imp_GetCurrentThreadId   0000000180004088     kernel32:KERNEL32.dll
 0002:00000090       __imp_GetSystemTimeAsFileTime 0000000180004090     kernel32:KERNEL32.dll
 0002:00000098       __imp_DisableThreadLibraryCalls 0000000180004098     kernel32:KERNEL32.dll
 0002:000000a0       __imp_InitializeSListHead  00000001800040a0     kernel32:KERNEL32.dll
 0002:000000a8       \177KERNEL32_NULL_THUNK_DATA 00000001800040a8     kernel32:KERNEL32.dll
 0002:000000b0       __imp_memcpy               00000001800040b0     vcruntime:VCRUNTIME140.dll
 0002:000000b8       __imp_memset               00000001800040b8     vcruntime:VCRUNTIME140.dll
 0002:000000c0       __imp_strchr               00000001800040c0     vcruntime:VCRUNTIME140.dll
 0002:000000c8       __imp___C_specific_handler 00000001800040c8     vcruntime:VCRUNTIME140.dll
 0002:000000d0       __imp___std_type_info_destroy_list 00000001800040d0     vcruntime:VCRUNTIME140.dll
 0002:000000d8       \177VCRUNTIME140_NULL_THUNK_DATA 00000001800040d8     vcruntime:VCRUNTIME140.dll
 0002:000000e0       __imp__errno               00000001800040e0     ucrt:api-ms-win-crt-runtime-l1-1-0.dll
 0002:000000e8       __imp_exit                 00000001800040e8     ucrt:api-ms-win-crt-runtime-l1-1-0.dll
 0002:000000f0       __imp__cexit               00000001800040f0     ucrt:api-ms-win-crt-runtime-l1-1-0.dll
 0002:000000f8       __imp__crt_atexit          00000001800040f8     ucrt:api-ms-win-crt-runtime-l1-1-0.dll
 0002:00000100       __imp__execute_onexit_table 0000000180004100     ucrt:api-ms-win-crt-runtime-l1-1-0.dll
 0002:00000108       __imp__register_onexit_function 0000000180004108     ucrt:api-ms-win-crt-runtime-l1-1-0.dll
 0002:00000110       __imp__initialize_onexit_table 0000000180004110     ucrt:api-ms-win-crt-runtime-l1-1-0.dll
 0002:00000118       __imp__initialize_narrow_environment 0000000180004118     ucrt:api-ms-win-crt-runtime-l1-1-0.dll
 0002:00000120       __imp__configure_narrow_argv 0000000180004120     ucrt:api-ms-win-crt-runtime-l1-1-0.dll
 0002:00000128       __imp__seh_filter_dll      0000000180004128     ucrt:api-ms-win-crt-runtime-l1-1-0.dll
 0002:00000130       __imp__initterm_e          0000000180004130     ucrt:api-ms-win-crt-runtime-l1-1-0.dll
 0002:00000138       __imp__initterm            0000000180004138     ucrt:api-ms-win-crt-runtime-l1-1-0.dll
 0002:00000140       \177api-ms-win-crt-runtime-l1-1-0_NULL_THUNK_DATA 0000000180004140     ucrt:api-ms-win-crt-runtime-l1-1-0.dll
 0002:00000148       __imp___acrt_iob_func      0000000180004148     ucrt:api-ms-win-crt-stdio-l1-1-0.dll
 0002:00000150       __imp_fflush               0000000180004150     ucrt:api-ms-win-crt-stdio-l1-1-0.dll
 0002:00000158       __imp___stdio_common_vsprintf 0000000180004158     ucrt:api-ms-win-crt-stdio-l1-1-0.dll
 0002:00000160       __imp___stdio_common_vfprintf 0000000180004160     ucrt:api-ms-win-crt-stdio-l1-1-0.dll
 0002:00000168       \177api-ms-win-crt-stdio-l1-1-0_NULL_THUNK_DATA 0000000180004168     ucrt:api-ms-win-crt-stdio-l1-1-0.dll
 0002:00000170       __imp_strcmp               0000000180004170     ucrt:api-ms-win-crt-string-l1-1-0.dll
 0002:00000178       __imp__strdup              0000000180004178     ucrt:api-ms-win-crt-string-l1-1-0.dll
 0002:00000178       __imp_strdup               0000000180004178     ucrt:api-ms-win-crt-string-l1-1-0.dll
 0002:00000180       __imp_strlen               0000000180004180     ucrt:api-ms-win-crt-string-l1-1-0.dll
 0002:00000188       __imp_strncpy              0000000180004188     ucrt:api-ms-win-crt-string-l1-1-0.dll
 0002:00000190       \177api-ms-win-crt-string-l1-1-0_NULL_THUNK_DATA 0000000180004190     ucrt:api-ms-win-crt-string-l1-1-0.dll
 0002:00000198       __guard_check_icall_fptr   0000000180004198     MSVCRT:guard_support.obj
 0002:000001a0       __guard_xfg_check_icall_fptr 00000001800041a0     MSVCRT:guard_support.obj
 0002:000001a8       __guard_dispatch_icall_fptr 00000001800041a8     MSVCRT:guard_support.obj
 0002:000001b0       __guard_xfg_dispatch_icall_fptr 00000001800041b0     MSVCRT:guard_support.obj
 0002:000001b8       __guard_xfg_table_dispatch_icall_fptr 00000001800041b8     MSVCRT:guard_support.obj
 0002:000001c0       __castguard_check_failure_os_handled_fptr 00000001800041c0     MSVCRT:guard_support.obj
 0002:000001c8       __guard_memcpy_fptr        00000001800041c8     vcruntime:softmemtag.obj
 0002:000001d0       __xc_a                     00000001800041d0     MSVCRT:initializers.obj
 0002:000001d8       __xc_z                     00000001800041d8     MSVCRT:initializers.obj
 0002:000001e0       __xi_a                     00000001800041e0     MSVCRT:initializers.obj
 0002:000001f0       __xi_z                     00000001800041f0     MSVCRT:initializers.obj
 0002:000001f8       __xl_a                     00000001800041f8     MSVCRT:tlssup.obj
 0002:00000200       __xl_z                     0000000180004200     MSVCRT:tlssup.obj
 0002:00000208       __xp_a                     0000000180004208     MSVCRT:initializers.obj
 0002:00000210       __xp_z                     0000000180004210     MSVCRT:initializers.obj
 0002:00000218       __xt_a                     0000000180004218     MSVCRT:initializers.obj
 0002:00000220       __xt_z                     0000000180004220     MSVCRT:initializers.obj
 0002:00000230       g_refKindStr               0000000180004230     libgetvern001.obj
 0002:000003e0       ??_C@_09BPLDFGCI@unknown_0@ 00000001800043e0     libgetvern001.obj
 0002:000003f0       ??_C@_0BL@FPNMECJD@JVMTI_HEAP_REFERENCE_CLASS@ 00000001800043f0     libgetvern001.obj
 0002:00000410       ??_C@_0BL@FKGKKLNM@JVMTI_HEAP_REFERENCE_FIELD@ 0000000180004410     libgetvern001.obj
 0002:00000430       ??_C@_0CD@CAEHCFJF@JVMTI_HEAP_REFERENCE_ARRAY_ELEM@ 0000000180004430     libgetvern001.obj
 0002:00000458       ??_C@_0CC@DNEBMCNK@JVMTI_HEAP_REFERENCE_CLASS_LOAD@ 0000000180004458     libgetvern001.obj
 0002:00000480       ??_C@_0BN@CJMIPEBB@JVMTI_HEAP_REFERENCE_SIGNERS@ 0000000180004480     libgetvern001.obj
 0002:000004a0       ??_C@_0CH@HBOIDPEB@JVMTI_HEAP_REFERENCE_PROTECTION@ 00000001800044a0     libgetvern001.obj
 0002:000004c8       ??_C@_0BP@MDKGDGKL@JVMTI_HEAP_REFERENCE_INTERFACE@ 00000001800044c8     libgetvern001.obj
 0002:000004e8       ??_C@_0CC@JJMIHNJH@JVMTI_HEAP_REFERENCE_STATIC_FIE@ 00000001800044e8     libgetvern001.obj
 0002:00000510       ??_C@_0CD@IDHEEGID@JVMTI_HEAP_REFERENCE_CONSTANT_P@ 0000000180004510     libgetvern001.obj
 0002:00000538       ??_C@_0CA@EFFCHNG@JVMTI_HEAP_REFERENCE_SUPERCLASS@ 0000000180004538     libgetvern001.obj
 0002:00000558       ??_C@_0L@PCDFHGCJ@unknown_11@ 0000000180004558     libgetvern001.obj
 0002:00000568       ??_C@_0L@NJBICFOK@unknown_12@ 0000000180004568     libgetvern001.obj
 0002:00000578       ??_C@_0L@MAADBEKL@unknown_13@ 0000000180004578     libgetvern001.obj
 0002:00000588       ??_C@_0L@IPECICGM@unknown_14@ 0000000180004588     libgetvern001.obj
 0002:00000598       ??_C@_0L@JGFJLDCN@unknown_15@ 0000000180004598     libgetvern001.obj
 0002:000005a8       ??_C@_0L@LNHEOAOO@unknown_16@ 00000001800045a8     libgetvern001.obj
 0002:000005b8       ??_C@_0L@KEGPNBKP@unknown_17@ 00000001800045b8     libgetvern001.obj
 0002:000005c8       ??_C@_0L@CDPHMNGA@unknown_18@ 00000001800045c8     libgetvern001.obj
 0002:000005d8       ??_C@_0L@DKOMPMCB@unknown_19@ 00000001800045d8     libgetvern001.obj
 0002:000005e8       ??_C@_0L@OJGIPJDB@unknown_20@ 00000001800045e8     libgetvern001.obj
 0002:000005f8       ??_C@_0CA@KAOFNDEM@JVMTI_HEAP_REFERENCE_JNI_GLOBAL@ 00000001800045f8     libgetvern001.obj
 0002:00000618       ??_C@_0CC@HPFAJBK@JVMTI_HEAP_REFERENCE_SYSTEM_CLA@ 0000000180004618     libgetvern001.obj
 0002:00000640       ??_C@_0BN@FDEGFOHC@JVMTI_HEAP_REFERENCE_MONITOR@ 0000000180004640     libgetvern001.obj
 0002:00000660       ??_C@_0CB@HKIBCMAJ@JVMTI_HEAP_REFERENCE_STACK_LOCA@ 0000000180004660     libgetvern001.obj
 0002:00000688       ??_C@_0BP@EAACMMOE@JVMTI_HEAP_REFERENCE_JNI_LOCAL@ 0000000180004688     libgetvern001.obj
 0002:000006a8       ??_C@_0BM@IJDEOGOE@JVMTI_HEAP_REFERENCE_THREAD@ 00000001800046a8     libgetvern001.obj
 0002:000006c8       ??_C@_0BL@EDGPPKC@JVMTI_HEAP_REFERENCE_OTHER@ 00000001800046c8     libgetvern001.obj
 0002:000006e4       ??_C@_04BCJPDBDA@Code@     00000001800046e4     libgetvern001.obj
 0002:000006f0       ??_C@_0BA@OCLMCFKC@LineNumberTable@ 00000001800046f0     libgetvern001.obj
 0002:00000700       ??_C@_0BD@CPAEPILC@LocalVariableTable@ 0000000180004700     libgetvern001.obj
 0002:00000718       ??_C@_0BH@NMBDNHBD@LocalVariableTypeTable@ 0000000180004718     libgetvern001.obj
 0002:00000730       ??_C@_0O@HIHEEDNJ@StackMapTable@ 0000000180004730     libgetvern001.obj
 0002:00000740       ??_C@_0L@HCDIAMJG@?9?5?$CFs?0?5?$CFd?3?5@ 0000000180004740     libgetvern001.obj
 0002:00000750       ??_C@_0JI@HLPECLFI@?$CD?5?4?4?4?6?$CD?5ERROR?3?5too?5many?5complai@ 0000000180004750     libgetvern001.obj
 0002:000007f0       ??_C@_0ED@JNEKCCOB@The?5following?5fake?5exception?5st@ 00000001800047f0     libgetvern001.obj
 0002:00000838       ??_C@_0CN@FCNMDFBH@nsk?4share?4Fake_Exception_for_RU@ 0000000180004838     libgetvern001.obj
 0002:00000868       ??_C@_08PGFFNAEI@?$CI?$CFs?3?$CFd?$CJ?5@ 0000000180004868     libgetvern001.obj
 0002:00000878       ??_C@_0DP@IENMAEGI@s?2test?2hotspot?2jtreg?2vmTestbase@ 0000000180004878     libgetvern001.obj
 0002:000008b8       ??_C@_0BL@NDJLFFJB@?7at?5nsk_lvcomplain?$CI?$CFs?3?$CFd?$CJ?6@ 00000001800048b8     libgetvern001.obj
 0002:000008d8       ??_C@_0BC@JOOKAFKF@?$CD?5ERROR?3?5?$CFs?0?5?$CFd?3?5@ 00000001800048d8     libgetvern001.obj
 0002:000008f0       ??_C@_09KJEAHMEH@?$CD?5ERROR?3?5@ 00000001800048f0     libgetvern001.obj
 0002:000008fc       ??_C@_02GPIOPFAK@?$DO?$DO@ 00000001800048fc     libgetvern001.obj
 0002:00000900       ??_C@_02FODMEDOG@?$DM?$DM@ 0000000180004900     libgetvern001.obj
 0002:00000904       ??_C@_02DJGKEECL@?4?4@     0000000180004904     libgetvern001.obj
 0002:00000908       ??_C@_0O@CJPGJOAF@?9?5?$CFs?0?5?$CFd?3?5?$CFs?5@ 0000000180004908     libgetvern001.obj
 0002:00000918       ??_C@_0CB@IAKPDOIC@?$CD?5?5?5verified?5assertion?5is?5FALSE@ 0000000180004918     libgetvern001.obj
 0002:00000940       ??_C@_0CO@LGONDEPD@stdout?3?5fflush?5failed?5?9?5err?$DN?$CFd?5@ 0000000180004940     libgetvern001.obj
 0002:00000970       ??_C@_0CO@KBGKJPBD@stderr?3?5fflush?5failed?5?9?5err?$DN?$CFd?5@ 0000000180004970     libgetvern001.obj
 0002:000009a0       ??_C@_0BB@JCNMKLLK@JVMTI_ERROR_NONE@ 00000001800049a0     libgetvern001.obj
 0002:000009b8       ??_C@_0BL@LDIMKLPH@JVMTI_ERROR_INVALID_THREAD@ 00000001800049b8     libgetvern001.obj
 0002:000009d8       ??_C@_0CB@PJFPAIKJ@JVMTI_ERROR_INVALID_THREAD_GROU@ 00000001800049d8     libgetvern001.obj
 0002:00000a00       ??_C@_0BN@LLMKHMNF@JVMTI_ERROR_INVALID_PRIORITY@ 0000000180004a00     libgetvern001.obj
 0002:00000a20       ??_C@_0CB@MBOFKAGB@JVMTI_ERROR_THREAD_NOT_SUSPENDE@ 0000000180004a20     libgetvern001.obj
 0002:00000a48       ??_C@_0BN@FABOLPBI@JVMTI_ERROR_THREAD_SUSPENDED@ 0000000180004a48     libgetvern001.obj
 0002:00000a68       ??_C@_0BN@FDGNOBJM@JVMTI_ERROR_THREAD_NOT_ALIVE@ 0000000180004a68     libgetvern001.obj
 0002:00000a88       ??_C@_0BL@GOBIFKNJ@JVMTI_ERROR_INVALID_OBJECT@ 0000000180004a88     libgetvern001.obj
 0002:00000aa8       ??_C@_0BK@FCMAJPPC@JVMTI_ERROR_INVALID_CLASS@ 0000000180004aa8     libgetvern001.obj
 0002:00000ac8       ??_C@_0BP@IKLLBKEB@JVMTI_ERROR_CLASS_NOT_PREPARED@ 0000000180004ac8     libgetvern001.obj
 0002:00000ae8       ??_C@_0BN@KLPPLKG@JVMTI_ERROR_INVALID_METHODID@ 0000000180004ae8     libgetvern001.obj
 0002:00000b08       ??_C@_0BN@BCEKOKND@JVMTI_ERROR_INVALID_LOCATION@ 0000000180004b08     libgetvern001.obj
 0002:00000b28       ??_C@_0BM@DFDGPME@JVMTI_ERROR_INVALID_FIELDID@ 0000000180004b28     libgetvern001.obj
 0002:00000b48       ??_C@_0BL@NELIEPEC@JVMTI_ERROR_NO_MORE_FRAMES@ 0000000180004b48     libgetvern001.obj
 0002:00000b68       ??_C@_0BJ@BDBECFDM@JVMTI_ERROR_OPAQUE_FRAME@ 0000000180004b68     libgetvern001.obj
 0002:00000b88       ??_C@_0BK@MIIFNLOB@JVMTI_ERROR_TYPE_MISMATCH@ 0000000180004b88     libgetvern001.obj
 0002:00000ba8       ??_C@_0BJ@HPCAOILC@JVMTI_ERROR_INVALID_SLOT@ 0000000180004ba8     libgetvern001.obj
 0002:00000bc8       ??_C@_0BG@CHILOPNI@JVMTI_ERROR_DUPLICATE@ 0000000180004bc8     libgetvern001.obj
 0002:00000be0       ??_C@_0BG@DIEMLHKM@JVMTI_ERROR_NOT_FOUND@ 0000000180004be0     libgetvern001.obj
 0002:00000bf8       ??_C@_0BM@NHMCKHOB@JVMTI_ERROR_INVALID_MONITOR@ 0000000180004bf8     libgetvern001.obj
 0002:00000c18       ??_C@_0BO@PPEDAJGL@JVMTI_ERROR_NOT_MONITOR_OWNER@ 0000000180004c18     libgetvern001.obj
 0002:00000c38       ??_C@_0BG@FCAIPEID@JVMTI_ERROR_INTERRUPT@ 0000000180004c38     libgetvern001.obj
 0002:00000c50       ??_C@_0CB@EGDBNKOI@JVMTI_ERROR_INVALID_CLASS_FORMA@ 0000000180004c50     libgetvern001.obj
 0002:00000c78       ??_C@_0CG@DGKOGIAL@JVMTI_ERROR_CIRCULAR_CLASS_DEFI@ 0000000180004c78     libgetvern001.obj
 0002:00000ca0       ??_C@_0BP@ICEALPKC@JVMTI_ERROR_FAILS_VERIFICATION@ 0000000180004ca0     libgetvern001.obj
 0002:00000cc0       ??_C@_0DC@JDACLMIO@JVMTI_ERROR_UNSUPPORTED_REDEFIN@ 0000000180004cc0     libgetvern001.obj
 0002:00000cf8       ??_C@_0DE@GKDKNOMJ@JVMTI_ERROR_UNSUPPORTED_REDEFIN@ 0000000180004cf8     libgetvern001.obj
 0002:00000d30       ??_C@_0BO@LAFKIOG@JVMTI_ERROR_INVALID_TYPESTATE@ 0000000180004d30     libgetvern001.obj
 0002:00000d50       ??_C@_0DH@INDGCLLB@JVMTI_ERROR_UNSUPPORTED_REDEFIN@ 0000000180004d50     libgetvern001.obj
 0002:00000d88       ??_C@_0DE@NHEOMMGI@JVMTI_ERROR_UNSUPPORTED_REDEFIN@ 0000000180004d88     libgetvern001.obj
 0002:00000dc0       ??_C@_0CA@EKPNJOEP@JVMTI_ERROR_UNSUPPORTED_VERSION@ 0000000180004dc0     libgetvern001.obj
 0002:00000de0       ??_C@_0BN@OFFMAHHL@JVMTI_ERROR_NAMES_DONT_MATCH@ 0000000180004de0     libgetvern001.obj
 0002:00000e00       ??_C@_0DN@HHBBLAKE@JVMTI_ERROR_UNSUPPORTED_REDEFIN@ 0000000180004e00     libgetvern001.obj
 0002:00000e40       ??_C@_0DO@HMBGBGNA@JVMTI_ERROR_UNSUPPORTED_REDEFIN@ 0000000180004e40     libgetvern001.obj
 0002:00000e80       ??_C@_0BP@PBECGKHJ@JVMTI_ERROR_UNMODIFIABLE_CLASS@ 0000000180004e80     libgetvern001.obj
 0002:00000ea0       ??_C@_0BK@CANILEHF@JVMTI_ERROR_NOT_AVAILABLE@ 0000000180004ea0     libgetvern001.obj
 0002:00000ec0       ??_C@_0CE@INJKMEFK@JVMTI_ERROR_MUST_POSSESS_CAPABI@ 0000000180004ec0     libgetvern001.obj
 0002:00000ee8       ??_C@_0BJ@LBFPFPDM@JVMTI_ERROR_NULL_POINTER@ 0000000180004ee8     libgetvern001.obj
 0002:00000f08       ??_C@_0BP@CHJPNNEM@JVMTI_ERROR_ABSENT_INFORMATION@ 0000000180004f08     libgetvern001.obj
 0002:00000f28       ??_C@_0BP@OMFMNLC@JVMTI_ERROR_INVALID_EVENT_TYPE@ 0000000180004f28     libgetvern001.obj
 0002:00000f48       ??_C@_0BN@BIBNPHHO@JVMTI_ERROR_ILLEGAL_ARGUMENT@ 0000000180004f48     libgetvern001.obj
 0002:00000f68       ??_C@_0BK@KKNDHDCE@JVMTI_ERROR_NATIVE_METHOD@ 0000000180004f68     libgetvern001.obj
 0002:00000f88       ??_C@_0BK@PMKCFHAE@JVMTI_ERROR_OUT_OF_MEMORY@ 0000000180004f88     libgetvern001.obj
 0002:00000fa8       ??_C@_0BK@NNJBDMNB@JVMTI_ERROR_ACCESS_DENIED@ 0000000180004fa8     libgetvern001.obj
 0002:00000fc8       ??_C@_0BI@GHECLMNC@JVMTI_ERROR_WRONG_PHASE@ 0000000180004fc8     libgetvern001.obj
 0002:00000fe0       ??_C@_0BF@OLIHJOII@JVMTI_ERROR_INTERNAL@ 0000000180004fe0     libgetvern001.obj
 0002:00000ff8       ??_C@_0BO@EOHGKJHI@JVMTI_ERROR_UNATTACHED_THREAD@ 0000000180004ff8     libgetvern001.obj
 0002:00001018       ??_C@_0CA@LKHFDACL@JVMTI_ERROR_INVALID_ENVIRONMENT@ 0000000180005018     libgetvern001.obj
 0002:00001038       ??_C@_0BA@MMFHLOKK@?$DMunknown?5error?$DO@ 0000000180005038     libgetvern001.obj
 0002:00001048       ??_C@_0CF@CBHOKDB@throwable?5?$DN?5jni?9?$DOExceptionOccur@ 0000000180005048     libgetvern001.obj
 0002:00001070       ??_C@_03OFAPEBGM@?$CFs?6@  0000000180005070     libgetvern001.obj
 0002:00001078       ??_C@_0DM@LPIGEGNJ@s?2test?2hotspot?2jtreg?2vmTestbase@ 0000000180005078     libgetvern001.obj
 0002:000010b8       ??_C@_0CC@NFCNPEPK@Exception?5in?5JNI?5call?5?$CIcleared?$CJ@ 00000001800050b8     libgetvern001.obj
 0002:000010e0       ??_C@_0BJ@IBAKFIKF@jni?9?$DOExceptionDescribe?$CI?$CJ@ 00000001800050e0     libgetvern001.obj
 0002:00001100       ??_C@_0BG@GGKALKMH@jni?9?$DOExceptionClear?$CI?$CJ@ 0000000180005100     libgetvern001.obj
 0002:00001118       ??_C@_0CF@JMGFGJLJ@?$CD?5?5?5verified?5JNI?5assertion?5is?5F@ 0000000180005118     libgetvern001.obj
 0002:00001140       ??_C@_0CB@MLNJNCLJ@?5?5jvmti?5error?3?5code?$DN?$CFd?0?5name?$DN?$CFs@ 0000000180005140     libgetvern001.obj
 0002:00001168       ??_C@_0CD@OHBGDKMK@?$CD?5?5?5jvmti?5error?3?5code?$DN?$CFd?0?5name?$DN@ 0000000180005168     libgetvern001.obj
 0002:00001190       ??_C@_0CG@JNNCGPHB@?$CD?5?5?5error?5expected?3?5code?$DN?$CFd?0?5na@ 0000000180005190     libgetvern001.obj
 0002:000011c0       ??_C@_0EB@IMGKPCGE@?$CIstr_obj?5?$DN?5jni?9?$DONewStringUTF?$CIco@ 00000001800051c0     libgetvern001.obj
 0002:00001210       ??_C@_0EA@HFOGGBCC@s?2test?2hotspot?2jtreg?2vmTestbase@ 0000000180005210     libgetvern001.obj
 0002:00001250       ??_C@_05KKCIMGE@error@     0000000180005250     libgetvern001.obj
 0002:00001258       ??_C@_0CJ@JACLEAA@Test?5failed?5by?5setFailStatus?$CI?$CJ?4@ 0000000180005258     libgetvern001.obj
 0002:00001290       ??_C@_0EA@PNBCDMOA@s?2test?2hotspot?2jtreg?2vmTestbase@ 0000000180005290     libgetvern001.obj
 0002:000012d0       ??_C@_0DI@ILAHDLMP@?$CI?$CKagentThreadProc?$CJ?$CIjvmti_env?0?5a@ 00000001800052d0     libgetvern001.obj
 0002:00001308       ??_C@_0BD@KDBALNLB@JVMTI?5agent?5thread@ 0000000180005308     libgetvern001.obj
 0002:00001320       ??_C@_0BB@NOKBFPFO@java?1lang?1Thread@ 0000000180005320     libgetvern001.obj
 0002:00001334       ??_C@_06FALKBLGB@?$DMinit?$DO@ 0000000180005334     libgetvern001.obj
 0002:00001340       ??_C@_0BG@IKDDPPGD@?$CILjava?1lang?1String?$DL?$CJV@ 0000000180005340     libgetvern001.obj
 0002:00001360       ??_C@_0EB@IFJBFEKC@?$CIthreadClass?5?$DN?5jni_env?9?$DOFindCla@ 0000000180005360     libgetvern001.obj
 0002:000013b0       ??_C@_0GF@FGFIBKKL@?$CIthreadCtor?5?$DN?5jni_env?9?$DOGetMetho@ 00000001800053b0     libgetvern001.obj
 0002:00001418       ??_C@_0DN@NCPDJLOG@?$CIthreadName?5?$DN?5jni_env?9?$DONewStrin@ 0000000180005418     libgetvern001.obj
 0002:00001460       ??_C@_0FE@PFKODBGC@?$CIthreadObject?5?$DN?5jni_env?9?$DONewObj@ 0000000180005460     libgetvern001.obj
 0002:000014c0       ??_C@_0ED@HOBAHHJI@?$CIthreadGlobalRef?5?$DN?5jni_env?9?$DONew@ 00000001800054c0     libgetvern001.obj
 0002:00001510       ??_C@_0FN@HNJJAHFC@jvmti_env?9?$DORunAgentThread?$CIagent@ 0000000180005510     libgetvern001.obj
 0002:00001570       ??_C@_0EA@MOJDNKDF@Debuggee?5status?5sync?5aborted?5be@ 0000000180005570     libgetvern001.obj
 0002:000015b0       ??_C@_0EA@EEOEJAEN@status?5?$DN?5syncDebuggeeStatus?$CIjni@ 00000001800055b0     libgetvern001.obj
 0002:000015f0       ??_C@_0BL@JBCFNBMB@nsk_jvmti_resetAgentData?$CI?$CJ@ 00000001800055f0     libgetvern001.obj
 0002:00001610       ??_C@_0EL@LPBEELIP@s?2test?2hotspot?2jtreg?2vmTestbase@ 0000000180005610     libgetvern001.obj
 0002:00001660       ??_C@_0CK@JDAMFDMJ@jvmti?9?$DOSetTag?$CIo?0?5tag?$CJ?5?$DN?$DN?5JVMTI_@ 0000000180005660     libgetvern001.obj
 0002:00001690       ??_C@_0CC@DAMNHKNI@Can?8t?5set?5tag?5?$CFli?5for?5object?5?$CFl@ 0000000180005690     libgetvern001.obj
 0002:000016b8       ??_C@_0DL@HAJPNKEF@jvmti?9?$DOGetObjectHashCode?$CIo?0?5?$CGha@ 00000001800056b8     libgetvern001.obj
 0002:000016f8       ??_C@_0BL@JFPIEOBF@Can?8t?5get?5hash?5object?5?$CFlx?6@ 00000001800056f8     libgetvern001.obj
 0002:00001718       ??_C@_0BG@DICPHBKN@setTag?3?5?$CF08x?5?$DM?9?5?$CF?53li@ 0000000180005718     libgetvern001.obj
 0002:00001730       ??_C@_0DH@FCEEBDMJ@?$CIs?5?$DN?5jni?9?$DOGetStringUTFChars?$CIsIn@ 0000000180005730     libgetvern001.obj
 0002:00001768       ??_C@_0BJ@OKKGHDCN@Can?8t?5get?5string?5at?5?$CF?$CDp?6@ 0000000180005768     libgetvern001.obj
 0002:00001788       ??_C@_0BP@EKFLGGFJ@Can?8t?5get?5string?5at?5?$CF?$CDp?3?5null?6@ 0000000180005788     libgetvern001.obj
 0002:000017a8       ??_C@_06ICODBHCL@?5?1?1?5?$CFs@ 00000001800057a8     libgetvern001.obj
 0002:000017b0       ??_C@_0DB@KGFPLEGO@?$CIr?5?$DN?5jvmti?9?$DOGetTag?$CIo?0?5?$CGtag?$CJ?$CJ?5?$DN?$DN@ 00000001800057b0     libgetvern001.obj
 0002:000017e8       ??_C@_0CO@PDAGBCGJ@Can?8t?5GetTag?5for?5object?5?$CFlx?4?5Re@ 00000001800057e8     libgetvern001.obj
 0002:00001818       ??_C@_0CH@HPEODOHC@TEST_BUG?3?5Max?4?5number?5of?5refs?5r@ 0000000180005818     libgetvern001.obj
 0002:00001840       ??_C@_0DI@PHFCABIM@?$CIr?5?$DN?5jvmti?9?$DOGetTag?$CIfrom?0?5?$CGtagFr@ 0000000180005840     libgetvern001.obj
 0002:00001878       ??_C@_0DI@MDEGFNKD@TEST_BUG?3?5Can?8t?5GetTag?5for?5obje@ 0000000180005878     libgetvern001.obj
 0002:000018b0       ??_C@_0DE@MLELJAHM@?$CIr?5?$DN?5jvmti?9?$DOGetTag?$CIto?0?5?$CGtagTo?$CJ?$CJ@ 00000001800058b0     libgetvern001.obj
 0002:000018e8       ??_C@_09OPJEJKBL@printdump@ 00000001800058e8     libgetvern001.obj
 0002:000018f8       ??_C@_0CJ@KCDEKOCJ@Wrong?5result?5of?5a?5valid?5call?5to@ 00000001800058f8     libgetvern001.obj
 0002:00001928       ??_C@_0CH@CDOJMNAO@JVMTI?5client?5was?5not?5properly?5l@ 0000000180005928     libgetvern001.obj
 0002:00001950       ??_C@_0BK@FEHOGPIL@?$DO?$DO?$DO?5functional?5check?5?4?4?4?6@ 0000000180005950     libgetvern001.obj
 0002:00001970       ??_C@_0CO@LFFKCNO@?$CIGetVersionNumber?$CJ?5unexpected?5e@ 0000000180005970     libgetvern001.obj
 0002:000019a0       ??_C@_0BG@EDDIIOGO@JVMTI?5version?3?5?$CFd?4?$CFd?6@ 00000001800059a0     libgetvern001.obj
 0002:000019b8       ??_C@_0O@BHPJPDFF@?$DO?$DO?$DO?5?4?4?4?5done?6@ 00000001800059b8     libgetvern001.obj
 0002:000019c8       ??_C@_0BM@OIEHJFGB@?$DO?$DO?$DO?5null?5pointer?5check?5?4?4?4?6@ 00000001800059c8     libgetvern001.obj
 0002:000019e8       ??_C@_0DD@PINJNLML@Error?5expected?3?5JVMTI_ERROR_NUL@ 00000001800059e8     libgetvern001.obj
 0002:00001a30       ??_C@_1EC@JIJBPKFM@?$AAa?$AAp?$AAi?$AA?9?$AAm?$AAs?$AA?9?$AAw?$AAi?$AAn?$AA?9?$AAc?$AAo?$AAr?$AAe@ 0000000180005a30     MSVCRT:thread_safe_statics.obj
 0002:00001a78       ??_C@_1BK@MGMFAEKH@?$AAk?$AAe?$AAr?$AAn?$AAe?$AAl?$AA3?$AA2?$AA?4?$AAd?$AAl?$AAl@ 0000000180005a78     MSVCRT:thread_safe_statics.obj
 0002:00001a98       ??_C@_0BJ@JEBJOJFJ@SleepConditionVariableCS@ 0000000180005a98     MSVCRT:thread_safe_statics.obj
 0002:00001ab8       ??_C@_0BJ@PGPPEPCC@WakeAllConditionVariable@ 0000000180005ab8     MSVCRT:thread_safe_statics.obj
 0002:00001ad8       _pDefaultRawDllMain        0000000180005ad8     MSVCRT:dll_dllmain.obj
 0002:00001ad8       _pRawDllMain               0000000180005ad8     MSVCRT:dll_dllmain.obj
 0002:00001ae0       __xmm@ffffffffffffffffffffffffffffffff 0000000180005ae0     MSVCRT:utility.obj
 0002:00001af0       _load_config_used          0000000180005af0     MSVCRT:loadcfg.obj
 0002:00001d00       _tls_used                  0000000180005d00     MSVCRT:tlssup.obj
 0002:00001d28       __volatile_metadata        0000000180005d28     <linker-defined>
 0002:000020e8       __rtc_iaa                  00000001800060e8     MSVCRT:initsect.obj
 0002:000020f0       __rtc_izz                  00000001800060f0     MSVCRT:initsect.obj
 0002:000020f8       __rtc_taa                  00000001800060f8     MSVCRT:initsect.obj
 0002:00002100       __rtc_tzz                  0000000180006100     MSVCRT:initsect.obj
 0002:00002108       _tls_start                 0000000180006108     MSVCRT:tlssup.obj
 0002:0000210c       _Init_thread_epoch         000000018000610c     MSVCRT:thread_safe_statics.obj
 0002:00002110       _tls_end                   0000000180006110     MSVCRT:tlssup.obj
 0002:00002790       __IMPORT_DESCRIPTOR_KERNEL32 0000000180006790     kernel32:KERNEL32.dll
 0002:000027a4       __IMPORT_DESCRIPTOR_VCRUNTIME140 00000001800067a4     vcruntime:VCRUNTIME140.dll
 0002:000027b8       __IMPORT_DESCRIPTOR_api-ms-win-crt-runtime-l1-1-0 00000001800067b8     ucrt:api-ms-win-crt-runtime-l1-1-0.dll
 0002:000027cc       __IMPORT_DESCRIPTOR_api-ms-win-crt-stdio-l1-1-0 00000001800067cc     ucrt:api-ms-win-crt-stdio-l1-1-0.dll
 0002:000027e0       __IMPORT_DESCRIPTOR_api-ms-win-crt-string-l1-1-0 00000001800067e0     ucrt:api-ms-win-crt-string-l1-1-0.dll
 0002:000027f4       __NULL_IMPORT_DESCRIPTOR   00000001800067f4     kernel32:KERNEL32.dll
 0003:00000030       _Init_global_epoch         0000000180007030     MSVCRT:thread_safe_statics.obj
 0003:00000040       __security_cookie          0000000180007040     MSVCRT:gs_cookie.obj
 0003:00000048       __security_cookie_complement 0000000180007048     MSVCRT:gs_cookie.obj
 0003:00000050       __scrt_native_dllmain_reason 0000000180007050     MSVCRT:utility.obj
 0003:00000058       __isa_available            0000000180007058     MSVCRT:cpu_disp.obj
 0003:0000005c       __isa_enabled              000000018000705c     MSVCRT:cpu_disp.obj
 0003:00000060       __memset_fast_string_threshold 0000000180007060     MSVCRT:cpu_disp.obj
 0003:00000068       __memset_nt_threshold      0000000180007068     MSVCRT:cpu_disp.obj
 0003:00000070       __scrt_ucrt_dll_is_in_use  0000000180007070     MSVCRT:ucrt_stubs.obj
 0003:00000080       g_wrongHeapCallbacks       0000000180007080     libgetvern001.obj
 0003:00000100       g_szTagInfo                0000000180007100     libgetvern001.obj
 0003:00002040       g_tagFlags                 0000000180009040     libgetvern001.obj
 0003:00002428       g_refsToVerifyCnt          0000000180009428     libgetvern001.obj
 0003:0000242c       g_fakeUserData             000000018000942c     libgetvern001.obj
 0003:00002430       g_tagVisitCount            0000000180009430     libgetvern001.obj
 0003:000033d0       g_refsToVerify             000000018000a3d0     libgetvern001.obj
 0003:0001aad0       g_userDataError            0000000180021ad0     libgetvern001.obj
 0003:0001ac70       ?_OptionsStorage@?1??__local_stdio_printf_options@@9@4_KA 0000000180021c70     libgetvern001.obj
 0003:0001b238       _tls_index                 0000000180022238     MSVCRT:tlssup.obj
 0003:0001b240       __scrt_current_native_startup_state 0000000180022240     MSVCRT:utility.obj
 0003:0001b248       __scrt_native_startup_lock 0000000180022248     MSVCRT:utility.obj
 0003:0001b288       __scrt_debugger_hook_flag  0000000180022288     MSVCRT:utility_desktop.obj
 0003:0001b290       ?__type_info_root_node@@3U__type_info_node@@A 0000000180022290     MSVCRT:tncleanup.obj
 0003:0001b2a0       ?_OptionsStorage@?1??__local_stdio_scanf_options@@9@4_KA 00000001800222a0     MSVCRT:default_local_stdio_options.obj
 0003:0001b2a8       __favor                    00000001800222a8     MSVCRT:cpu_disp.obj
 0003:0001b2b0       __dyn_tls_init_callback    00000001800222b0     <common>

 entry point at        0001:000021f0

 Static symbols

 0000:fffdb000       .debug$S                   0000000180000000     getvern001.exp
 0000:fffdb000       .debug$S                   0000000180000000     vcruntime:VCRUNTIME140.dll
 0000:fffdb000       .debug$S                   0000000180000000     vcruntime:VCRUNTIME140.dll
 0000:fffdb000       .debug$S                   0000000180000000     vcruntime:VCRUNTIME140.dll
 0000:fffdb000       .debug$S                   0000000180000000     vcruntime:VCRUNTIME140.dll
 0000:fffdb000       .debug$S                   0000000180000000     vcruntime:VCRUNTIME140.dll
 0000:fffdb000       .debug$S                   0000000180000000     vcruntime:VCRUNTIME140.dll
 0000:fffdb000       .debug$S                   0000000180000000     vcruntime:VCRUNTIME140.dll
 0000:fffdb000       .debug$S                   0000000180000000     ucrt:api-ms-win-crt-convert-l1-1-0.dll
 0002:ffffc000       .idata$6                   0000000180000000     ucrt:api-ms-win-crt-convert-l1-1-0.dll
 0000:fffdb000       .debug$S                   0000000180000000     ucrt:api-ms-win-crt-heap-l1-1-0.dll
 0000:fffdb000       .debug$S                   0000000180000000     ucrt:api-ms-win-crt-heap-l1-1-0.dll
 0000:fffdb000       .debug$S                   0000000180000000     ucrt:api-ms-win-crt-heap-l1-1-0.dll
 0000:fffdb000       .debug$S                   0000000180000000     ucrt:api-ms-win-crt-heap-l1-1-0.dll
 0002:ffffc000       .idata$6                   0000000180000000     ucrt:api-ms-win-crt-heap-l1-1-0.dll
 0000:fffdb000       .debug$S                   0000000180000000     ucrt:api-ms-win-crt-runtime-l1-1-0.dll
 0000:fffdb000       .debug$S                   0000000180000000     ucrt:api-ms-win-crt-runtime-l1-1-0.dll
 0000:fffdb000       .debug$S                   0000000180000000     ucrt:api-ms-win-crt-runtime-l1-1-0.dll
 0000:fffdb000       .debug$S                   0000000180000000     ucrt:api-ms-win-crt-runtime-l1-1-0.dll
 0000:fffdb000       .debug$S                   0000000180000000     ucrt:api-ms-win-crt-runtime-l1-1-0.dll
 0000:fffdb000       .debug$S                   0000000180000000     ucrt:api-ms-win-crt-runtime-l1-1-0.dll
 0000:fffdb000       .debug$S                   0000000180000000     ucrt:api-ms-win-crt-runtime-l1-1-0.dll
 0000:fffdb000       .debug$S                   0000000180000000     ucrt:api-ms-win-crt-runtime-l1-1-0.dll
 0000:fffdb000       .debug$S                   0000000180000000     ucrt:api-ms-win-crt-runtime-l1-1-0.dll
 0000:fffdb000       .debug$S                   0000000180000000     ucrt:api-ms-win-crt-runtime-l1-1-0.dll
 0000:fffdb000       .debug$S                   0000000180000000     ucrt:api-ms-win-crt-runtime-l1-1-0.dll
 0000:fffdb000       .debug$S                   0000000180000000     ucrt:api-ms-win-crt-runtime-l1-1-0.dll
 0000:fffdb000       .debug$S                   0000000180000000     ucrt:api-ms-win-crt-runtime-l1-1-0.dll
 0000:fffdb000       .debug$S                   0000000180000000     ucrt:api-ms-win-crt-runtime-l1-1-0.dll
 0000:fffdb000       .debug$S                   0000000180000000     ucrt:api-ms-win-crt-runtime-l1-1-0.dll
 0000:fffdb000       .debug$S                   0000000180000000     ucrt:api-ms-win-crt-runtime-l1-1-0.dll
 0000:fffdb000       .debug$S                   0000000180000000     ucrt:api-ms-win-crt-stdio-l1-1-0.dll
 0000:fffdb000       .debug$S                   0000000180000000     ucrt:api-ms-win-crt-stdio-l1-1-0.dll
 0000:fffdb000       .debug$S                   0000000180000000     ucrt:api-ms-win-crt-stdio-l1-1-0.dll
 0000:fffdb000       .debug$S                   0000000180000000     ucrt:api-ms-win-crt-stdio-l1-1-0.dll
 0000:fffdb000       .debug$S                   0000000180000000     ucrt:api-ms-win-crt-stdio-l1-1-0.dll
 0000:fffdb000       .debug$S                   0000000180000000     ucrt:api-ms-win-crt-stdio-l1-1-0.dll
 0000:fffdb000       .debug$S                   0000000180000000     ucrt:api-ms-win-crt-stdio-l1-1-0.dll
 0000:fffdb000       .debug$S                   0000000180000000     ucrt:api-ms-win-crt-stdio-l1-1-0.dll
 0000:fffdb000       .debug$S                   0000000180000000     ucrt:api-ms-win-crt-stdio-l1-1-0.dll
 0000:fffdb000       .debug$S                   0000000180000000     ucrt:api-ms-win-crt-stdio-l1-1-0.dll
 0000:fffdb000       .debug$S                   0000000180000000     ucrt:api-ms-win-crt-string-l1-1-0.dll
 0000:fffdb000       .debug$S                   0000000180000000     ucrt:api-ms-win-crt-string-l1-1-0.dll
 0000:fffdb000       .debug$S                   0000000180000000     ucrt:api-ms-win-crt-string-l1-1-0.dll
 0000:fffdb000       .debug$S                   0000000180000000     ucrt:api-ms-win-crt-string-l1-1-0.dll
 0000:fffdb000       .debug$S                   0000000180000000     ucrt:api-ms-win-crt-string-l1-1-0.dll
 0000:fffdb000       .debug$S                   0000000180000000     ucrt:api-ms-win-crt-string-l1-1-0.dll
 0000:fffdb000       .debug$S                   0000000180000000     ucrt:api-ms-win-crt-string-l1-1-0.dll
 0000:fffdb000       .debug$S                   0000000180000000     ucrt:api-ms-win-crt-string-l1-1-0.dll
 0000:fffdb000       .debug$S                   0000000180000000     kernel32:KERNEL32.dll
 0000:fffdb000       .debug$S                   0000000180000000     kernel32:KERNEL32.dll
 0000:fffdb000       .debug$S                   0000000180000000     kernel32:KERNEL32.dll
 0000:fffdb000       .debug$S                   0000000180000000     kernel32:KERNEL32.dll
 0000:fffdb000       .debug$S                   0000000180000000     kernel32:KERNEL32.dll
 0000:fffdb000       .debug$S                   0000000180000000     kernel32:KERNEL32.dll
 0000:fffdb000       .debug$S                   0000000180000000     kernel32:KERNEL32.dll
 0000:fffdb000       .debug$S                   0000000180000000     kernel32:KERNEL32.dll
 0000:fffdb000       .debug$S                   0000000180000000     kernel32:KERNEL32.dll
 0000:fffdb000       .debug$S                   0000000180000000     kernel32:KERNEL32.dll
 0000:fffdb000       .debug$S                   0000000180000000     kernel32:KERNEL32.dll
 0000:fffdb000       .debug$S                   0000000180000000     kernel32:KERNEL32.dll
 0000:fffdb000       .debug$S                   0000000180000000     kernel32:KERNEL32.dll
 0000:fffdb000       .debug$S                   0000000180000000     kernel32:KERNEL32.dll
 0000:fffdb000       .debug$S                   0000000180000000     kernel32:KERNEL32.dll
 0000:fffdb000       .debug$S                   0000000180000000     kernel32:KERNEL32.dll
 0000:fffdb000       .debug$S                   0000000180000000     kernel32:KERNEL32.dll
 0000:fffdb000       .debug$S                   0000000180000000     kernel32:KERNEL32.dll
 0000:fffdb000       .debug$S                   0000000180000000     kernel32:KERNEL32.dll
 0000:fffdb000       .debug$S                   0000000180000000     kernel32:KERNEL32.dll
 0000:fffdb000       .debug$S                   0000000180000000     kernel32:KERNEL32.dll
 0000:fffdb000       .debug$S                   0000000180000000     kernel32:KERNEL32.dll
 0000:fffdb000       .debug$S                   0000000180000000     kernel32:KERNEL32.dll
 0000:fffdb000       .debug$S                   0000000180000000     kernel32:KERNEL32.dll
 0000:fffdb000       .debug$S                   0000000180000000     kernel32:KERNEL32.dll
 0000:fffdb000       .debug$S                   0000000180000000     kernel32:KERNEL32.dll
 0000:fffdb000       .debug$S                   0000000180000000     kernel32:KERNEL32.dll
 0000:fffdb000       .debug$S                   0000000180000000     kernel32:KERNEL32.dll
 0001:00000e0c       addRefToVerify             0000000180001e0c f   libgetvern001.obj
 0001:00000e78       agentThreadWrapper         0000000180001e78 f   libgetvern001.obj
 0001:00001068       file_basename              0000000180002068 f   libgetvern001.obj
 0001:000016d4       startAgentThreadWrapper    00000001800026d4 f   libgetvern001.obj
 0001:00001a14       syncDebuggeeStatus         0000000180002a14 f   libgetvern001.obj
 0001:00001cb4       capture_previous_context   0000000180002cb4 f   MSVCRT:gs_report.obj
 0001:00001d28       ?__scrt_initialize_thread_safe_statics@@YAHXZ 0000000180002d28 f   MSVCRT:thread_safe_statics.obj
 0001:00001df8       ?__scrt_uninitialize_thread_safe_statics@@YAXXZ 0000000180002df8 f   MSVCRT:thread_safe_statics.obj
 0001:00001ea0       $$000000                   0000000180002ea0     MSVCRT:amdsecgs.obj
 0001:00001ed0       ?dllmain_crt_dispatch@@YAHQEAUHINSTANCE__@@KQEAX@Z 0000000180002ed0 f   MSVCRT:dll_dllmain.obj
 0001:00001f20       ?dllmain_crt_process_attach@@YAHQEAUHINSTANCE__@@QEAX@Z 0000000180002f20 f   MSVCRT:dll_dllmain.obj
 0001:00002038       ?dllmain_crt_process_detach@@YAH_N@Z 0000000180003038 f   MSVCRT:dll_dllmain.obj
 0001:000020bc       ?dllmain_dispatch@@YAHQEAUHINSTANCE__@@KQEAX@Z 00000001800030bc f   MSVCRT:dll_dllmain.obj
 0001:00002ad0       $$000000                   0000000180003ad0     MSVCRT:guard_dispatch.obj
 0001:00002af0       $$000000                   0000000180003af0     MSVCRT:guard_xfg_dispatch.obj
 0001:00002b06       ?fin$0@?0??dllmain_crt_process_attach@@YAHQEAUHINSTANCE__@@QEAX@Z@4HA 0000000180003b06 f   MSVCRT:dll_dllmain.obj
 0001:00002b1d       ?fin$0@?0??dllmain_crt_process_detach@@YAH_N@Z@4HA 0000000180003b1d f   MSVCRT:dll_dllmain.obj
 0001:00002b36       ?fin$1@?0??dllmain_crt_process_detach@@YAH_N@Z@4HA 0000000180003b36 f   MSVCRT:dll_dllmain.obj
 0001:00002b4a       ?filt$0@?0??dllmain_dispatch@@YAHQEAUHINSTANCE__@@KQEAX@Z@4HA 0000000180003b4a f   MSVCRT:dll_dllmain.obj
 0001:00002b80       __scrt_is_nonwritable_in_current_image$filt$0 0000000180003b80 f   MSVCRT:utility.obj
 0002:000001e8       ?__scrt_initialize_tss_var@@3P6AHXZEA 00000001800041e8     MSVCRT:thread_safe_statics.obj
 0002:00000310       ?opcLengths@@3QBEB         0000000180004310     libgetvern001.obj
 0002:00001a20       GS_ExceptionPointers       0000000180005a20     MSVCRT:gs_report.obj
 0002:00002118       $unwind$fprintf            0000000180006118     libgetvern001.obj
 0002:00002124       $unwind$printf             0000000180006124     libgetvern001.obj
 0002:00002130       $unwind$?NewObject@JNIEnv_@@QEAAPEAV_jobject@@PEAV_jclass@@PEAU_jmethodID@@ZZ 0000000180006130     libgetvern001.obj
 0002:00002130       $unwind$nsk_lcomplain      0000000180006130     libgetvern001.obj
 0002:00002130       $unwind$nsk_ldisplay       0000000180006130     libgetvern001.obj
 0002:00002138       $unwind$nsk_lvdisplay      0000000180006138     libgetvern001.obj
 0002:00002138       $unwind$_RTC_Initialize    0000000180006138     MSVCRT:initsect.obj
 0002:00002138       $unwind$_RTC_Terminate     0000000180006138     MSVCRT:initsect.obj
 0002:00002138       $unwind$?__scrt_initialize_thread_safe_statics@@YAHXZ 0000000180006138     MSVCRT:thread_safe_statics.obj
 0002:00002144       $unwind$nsk_lvcomplain     0000000180006144     libgetvern001.obj
 0002:0000215c       $unwind$nsk_ltrace         000000018000615c     libgetvern001.obj
 0002:0000215c       $unwind$__report_gsfailure 000000018000615c     MSVCRT:gs_report.obj
 0002:00002164       $unwind$Agent_Initialize   0000000180006164     libgetvern001.obj
 0002:00002164       $unwind$Java_nsk_jvmti_GetVersionNumber_getvern001_check 0000000180006164     libgetvern001.obj
 0002:00002164       $unwind$nsk_lvtrace        0000000180006164     libgetvern001.obj
 0002:00002164       $unwind$__raise_securityfailure 0000000180006164     MSVCRT:gs_report.obj
 0002:00002164       $unwind$__scrt_initialize_crt 0000000180006164     MSVCRT:utility.obj
 0002:00002164       $unwind$__scrt_initialize_onexit_tables 0000000180006164     MSVCRT:utility.obj
 0002:00002164       $unwind$__scrt_release_startup_lock 0000000180006164     MSVCRT:utility.obj
 0002:00002164       $unwind$__scrt_uninitialize_crt 0000000180006164     MSVCRT:utility.obj
 0002:00002164       $unwind$_onexit            0000000180006164     MSVCRT:utility.obj
 0002:0000216c       $unwind$nsk_lverify        000000018000616c     libgetvern001.obj
 0002:0000217c       $unwind$nsk_vprintf        000000018000617c     libgetvern001.obj
 0002:0000218c       $unwind$nsk_printf         000000018000618c     libgetvern001.obj
 0002:00002194       $unwind$?nsk_jni_lverify@@YAHHPEAUJNIEnv_@@HQEBDH1ZZ 0000000180006194     libgetvern001.obj
 0002:000021a8       $unwind$?nsk_jni_check_exception@@YAHPEAUJNIEnv_@@QEBDH@Z 00000001800061a8     libgetvern001.obj
 0002:000021c4       $unwind$Java_nsk_jvmti_unit_FollowReferences_FollowRefObjects_resetTags 00000001800061c4     libgetvern001.obj
 0002:000021c4       $unwind$addRefToVerify     00000001800061c4     libgetvern001.obj
 0002:000021c4       $unwind$nsk_jvmti_resetAgentData 00000001800061c4     libgetvern001.obj
 0002:000021c4       $unwind$nsk_jvmti_setFailStatus 00000001800061c4     libgetvern001.obj
 0002:000021c4       $unwind$__scrt_initialize_default_local_stdio_options 00000001800061c4     MSVCRT:default_local_stdio_options.obj
 0002:000021c4       $unwind$?dllmain_crt_dispatch@@YAHQEAUHINSTANCE__@@KQEAX@Z 00000001800061c4     MSVCRT:dll_dllmain.obj
 0002:000021c4       $unwind$DllMain            00000001800061c4     MSVCRT:dll_dllmain_stub.obj
 0002:000021c4       $unwind$__GSHandlerCheck   00000001800061c4     MSVCRT:gshandler.obj
 0002:000021c4       $unwind$?__scrt_uninitialize_thread_safe_statics@@YAXXZ 00000001800061c4     MSVCRT:thread_safe_statics.obj
 0002:000021c4       $unwind$__scrt_acquire_startup_lock 00000001800061c4     MSVCRT:utility.obj
 0002:000021c4       $unwind$__scrt_dllmain_after_initialize_c 00000001800061c4     MSVCRT:utility.obj
 0002:000021c4       $unwind$__scrt_dllmain_before_initialize_c 00000001800061c4     MSVCRT:utility.obj
 0002:000021c4       $unwind$__scrt_dllmain_crt_thread_attach 00000001800061c4     MSVCRT:utility.obj
 0002:000021c4       $unwind$__scrt_dllmain_crt_thread_detach 00000001800061c4     MSVCRT:utility.obj
 0002:000021c4       $unwind$__scrt_dllmain_uninitialize_c 00000001800061c4     MSVCRT:utility.obj
 0002:000021c4       $unwind$__scrt_dllmain_uninitialize_critical 00000001800061c4     MSVCRT:utility.obj
 0002:000021c4       $unwind$atexit             00000001800061c4     MSVCRT:utility.obj
 0002:000021cc       $unwind$nsk_jvmti_lverify  00000001800061cc     libgetvern001.obj
 0002:000021e0       $unwind$exitOnError        00000001800061e0     libgetvern001.obj
 0002:000021f0       $unwind$Java_nsk_share_jvmti_ArgumentHandler_getAgentOptionsString 00000001800061f0     libgetvern001.obj
 0002:00002204       $unwind$Java_nsk_jvmti_unit_FollowReferences_FollowRefObjects_getTag 0000000180006204     libgetvern001.obj
 0002:00002204       $unwind$Java_nsk_share_jvmti_DebugeeClass_checkStatus 0000000180006204     libgetvern001.obj
 0002:00002204       $unwind$agentThreadWrapper 0000000180006204     libgetvern001.obj
 0002:00002214       $unwind$startAgentThreadWrapper 0000000180006214     libgetvern001.obj
 0002:00002230       $unwind$syncDebuggeeStatus 0000000180006230     libgetvern001.obj
 0002:00002230       $unwind$__scrt_dllmain_exception_filter 0000000180006230     MSVCRT:utility.obj
 0002:00002244       $unwind$Java_nsk_share_jvmti_DebugeeClass_resetAgentData 0000000180006244     libgetvern001.obj
 0002:0000224c       $unwind$MA_checkStatus     000000018000624c     libgetvern001.obj
 0002:00002260       $unwind$Java_nsk_jvmti_unit_FollowReferences_FollowRefObjects_setTag 0000000180006260     libgetvern001.obj
 0002:00002278       $unwind$Java_nsk_jvmti_unit_FollowReferences_FollowRefObjects_addRefToVerify 0000000180006278     libgetvern001.obj
 0002:00002294       $unwind$capture_previous_context 0000000180006294     MSVCRT:gs_report.obj
 0002:000022a0       $unwind$__GSHandlerCheckCommon 00000001800062a0     MSVCRT:gshandler.obj
 0002:000022a8       $xdatasym                  00000001800062a8     MSVCRT:amdsecgs.obj
 0002:000022ac       $unwind$?dllmain_crt_process_attach@@YAHQEAUHINSTANCE__@@QEAX@Z 00000001800062ac     MSVCRT:dll_dllmain.obj
 0002:000022e8       $unwind$?fin$0@?0??dllmain_crt_process_attach@@YAHQEAUHINSTANCE__@@QEAX@Z@4HA 00000001800062e8     MSVCRT:dll_dllmain.obj
 0002:000022e8       $unwind$?fin$0@?0??dllmain_crt_process_detach@@YAH_N@Z@4HA 00000001800062e8     MSVCRT:dll_dllmain.obj
 0002:000022e8       $unwind$?fin$1@?0??dllmain_crt_process_detach@@YAH_N@Z@4HA 00000001800062e8     MSVCRT:dll_dllmain.obj
 0002:000022f0       $unwind$?dllmain_crt_process_detach@@YAH_N@Z 00000001800062f0     MSVCRT:dll_dllmain.obj
 0002:00002344       $unwind$?dllmain_dispatch@@YAHQEAUHINSTANCE__@@KQEAX@Z 0000000180006344     MSVCRT:dll_dllmain.obj
 0002:0000236c       $unwind$?filt$0@?0??dllmain_dispatch@@YAHQEAUHINSTANCE__@@KQEAX@Z@4HA 000000018000636c     MSVCRT:dll_dllmain.obj
 0002:00002374       $unwind$_DllMainCRTStartup 0000000180006374     MSVCRT:dll_dllmain.obj
 0002:00002384       $unwind$__scrt_is_nonwritable_in_current_image 0000000180006384     MSVCRT:utility.obj
 0002:000023a4       $unwind$__scrt_is_nonwritable_in_current_image$filt$0 00000001800063a4     MSVCRT:utility.obj
 0002:000023ac       $unwind$__scrt_fastfail    00000001800063ac     MSVCRT:utility_desktop.obj
 0002:000023bc       $unwind$__security_init_cookie 00000001800063bc     MSVCRT:gs_support.obj
 0002:000023c8       $unwind$__isa_available_init 00000001800063c8     MSVCRT:cpu_disp.obj
 0002:000023d8       $xdatasym                  00000001800063d8     MSVCRT:guard_dispatch.obj
 0002:000023e0       $xdatasym                  00000001800063e0     MSVCRT:guard_xfg_dispatch.obj
 0002:000023f0       .edata                     00000001800063f0     getvern001.exp
 0002:00002418       rgpv                       0000000180006418     getvern001.exp
 0002:00002454       rgszName                   0000000180006454     getvern001.exp
 0002:00002490       rgwOrd                     0000000180006490     getvern001.exp
 0002:000024ae       szName                     00000001800064ae     getvern001.exp
 0002:000024bd       $N00001                    00000001800064bd     getvern001.exp
 0002:000024cc       $N00002                    00000001800064cc     getvern001.exp
 0002:000024d9       $N00003                    00000001800064d9     getvern001.exp
 0002:0000250a       $N00004                    000000018000650a     getvern001.exp
 0002:0000254f       $N00005                    000000018000654f     getvern001.exp
 0002:0000258c       $N00006                    000000018000658c     getvern001.exp
 0002:000025d4       $N00007                    00000001800065d4     getvern001.exp
 0002:00002614       $N00008                    0000000180006614     getvern001.exp
 0002:00002651       $N00009                    0000000180006651     getvern001.exp
 0002:0000268c       $N00010                    000000018000668c     getvern001.exp
 0002:000026ba       $N00011                    00000001800066ba     getvern001.exp
 0002:000026eb       $N00012                    00000001800066eb     getvern001.exp
 0002:0000271a       $N00013                    000000018000671a     getvern001.exp
 0002:00002749       $N00014                    0000000180006749     getvern001.exp
 0002:0000277e       $N00015                    000000018000677e     getvern001.exp
 0002:00002b8a       .idata$6                   0000000180006b8a     kernel32:KERNEL32.dll
 0002:00002bee       .idata$6                   0000000180006bee     vcruntime:VCRUNTIME140.dll
 0002:00002d5a       .idata$6                   0000000180006d5a     ucrt:api-ms-win-crt-runtime-l1-1-0.dll
 0002:00002d7c       .idata$6                   0000000180006d7c     ucrt:api-ms-win-crt-stdio-l1-1-0.dll
 0002:00002d9c       .idata$6                   0000000180006d9c     ucrt:api-ms-win-crt-string-l1-1-0.dll
 0003:00000000       ?codeAttributeName@@3PEBDEB 0000000180007000     libgetvern001.obj
 0003:00000008       ?lineNumberAttributeName@@3PEBDEB 0000000180007008     libgetvern001.obj
 0003:00000010       ?localVarAttributeName@@3PEBDEB 0000000180007010     libgetvern001.obj
 0003:00000018       ?localVarTypeAttributeName@@3PEBDEB 0000000180007018     libgetvern001.obj
 0003:00000020       ?stackMapAttributeName@@3PEBDEB 0000000180007020     libgetvern001.obj
 0003:00000028       ?callBytes@@3PAEA          0000000180007028     libgetvern001.obj
 0003:0000002c       ?allocBytes@@3PAEA         000000018000702c     libgetvern001.obj
 0003:0001aad4       redefineAttempted          0000000180021ad4     libgetvern001.obj
 0003:0001aad8       nsk_context                0000000180021ad8     libgetvern001.obj
 0003:0001aae4       redefineSucceed            0000000180021ae4     libgetvern001.obj
 0003:0001aae8       agentFailed                0000000180021ae8     libgetvern001.obj
 0003:0001aaec       currentAgentStatus         0000000180021aec     libgetvern001.obj
 0003:0001aaf0       context                    0000000180021af0     libgetvern001.obj
 0003:0001aba8       agentThread                0000000180021ba8     libgetvern001.obj
 0003:0001abb0       agentThreadProc            0000000180021bb0     libgetvern001.obj
 0003:0001abb8       agentThreadArg             0000000180021bb8     libgetvern001.obj
 0003:0001abc0       agent_data                 0000000180021bc0     libgetvern001.obj
 0003:0001abd0       jvmti_env                  0000000180021bd0     libgetvern001.obj
 0003:0001abd8       jvm                        0000000180021bd8     libgetvern001.obj
 0003:0001abe0       jni_env                    0000000180021be0     libgetvern001.obj
 0003:0001abe8       checkStatus_func           0000000180021be8     libgetvern001.obj
 0003:0001abf0       ?codeAttributeIndex@@3GA   0000000180021bf0     libgetvern001.obj
 0003:0001abf2       printdump                  0000000180021bf2     libgetvern001.obj
 0003:0001abf4       ?lineNumberAttributeIndex@@3GA 0000000180021bf4     libgetvern001.obj
 0003:0001abf8       ?localVarAttributeIndex@@3GA 0000000180021bf8     libgetvern001.obj
 0003:0001abfc       ?localVarTypeAttributeIndex@@3GA 0000000180021bfc     libgetvern001.obj
 0003:0001ac00       ?stackMapAttributeIndex@@3GA 0000000180021c00     libgetvern001.obj
 0003:0001ac04       ?stackFrameOffset@@3GA     0000000180021c04     libgetvern001.obj
 0003:0001ac08       ?mode@@3HA                 0000000180021c08     libgetvern001.obj
 0003:0001ac0c       ?constantPoolSize@@3GA     0000000180021c0c     libgetvern001.obj
 0003:0001ac10       ?orig@@3PEBEEB             0000000180021c10     libgetvern001.obj
 0003:0001ac18       ?gen@@3PEAEEA              0000000180021c18     libgetvern001.obj
 0003:0001ac20       ?inputPos@@3PEAEEA         0000000180021c20     libgetvern001.obj
 0003:0001ac28       ?endPos@@3PEBEEB           0000000180021c28     libgetvern001.obj
 0003:0001ac30       ?genPos@@3PEAEEA           0000000180021c30     libgetvern001.obj
 0003:0001ac38       ?markPos@@3PEAEEA          0000000180021c38     libgetvern001.obj
 0003:0001ac40       ?constantPool@@3PEAPEADEA  0000000180021c40     libgetvern001.obj
 0003:0001ac48       ?constantPoolCount@@3GA    0000000180021c48     libgetvern001.obj
 0003:0001ac4c       ?zeroBytes@@3PAEA          0000000180021c4c     libgetvern001.obj
 0003:0001ac50       ?codeLength@@3IA           0000000180021c50     libgetvern001.obj
 0003:0001ac54       result                     0000000180021c54     libgetvern001.obj
 0003:0001ac58       ?map@@3PEAIEA              0000000180021c58     libgetvern001.obj
 0003:0001ac60       ?widening@@3PEACEA         0000000180021c60     libgetvern001.obj
 0003:0001ac68       jvmti                      0000000180021c68     libgetvern001.obj
 0003:0001ac80       GS_ExceptionRecord         0000000180021c80     MSVCRT:gs_report.obj
 0003:0001ad20       GS_ContextRecord           0000000180021d20     MSVCRT:gs_report.obj
 0003:0001b1f0       ?g_tss_cv@@3U_RTL_CONDITION_VARIABLE@@A 00000001800221f0     MSVCRT:thread_safe_statics.obj
 0003:0001b1f8       ?g_tss_event@@3PEAXEA      00000001800221f8     MSVCRT:thread_safe_statics.obj
 0003:0001b200       ?g_tss_mutex@@3U_RTL_CRITICAL_SECTION@@A 0000000180022200     MSVCRT:thread_safe_statics.obj
 0003:0001b228       ?g_sleep_condition_variable_cs@@3P6AHPEAU_RTL_CONDITION_VARIABLE@@PEAU_RTL_CRITICAL_SECTION@@K@ZEA 0000000180022228     MSVCRT:thread_safe_statics.obj
 0003:0001b230       ?g_wake_all_condition_variable@@3P6AXPEAU_RTL_CONDITION_VARIABLE@@@ZEA 0000000180022230     MSVCRT:thread_safe_statics.obj
 0003:0001b23c       ?__proc_attached@@3HA      000000018002223c     MSVCRT:dll_dllmain.obj
 0003:0001b250       ?is_initialized_as_dll@@3_NA 0000000180022250     MSVCRT:utility.obj
 0003:0001b251       ?module_local_atexit_table_initialized@@3_NA 0000000180022251     MSVCRT:utility.obj
 0003:0001b258       ?module_local_atexit_table@@3U_onexit_table_t@@A 0000000180022258     MSVCRT:utility.obj
 0003:0001b270       ?module_local_at_quick_exit_table@@3U_onexit_table_t@@A 0000000180022270     MSVCRT:utility.obj
